:020000021000EC
:10F000004BC0000082C0000080C000007EC0000035
:10F010007CC000007AC0000078C0000076C000000C
:10F0200074C0000072C000009BC500006EC00000EC
:10F030006CC000006AC0000068C0000066C000002C
:10F0400064C0000062C0000060C000005EC000003C
:10F05000E4C100005AC0000058C0000056C00000C3
:10F0600054C0000052C0000050C000004EC000005C
:10F070004CC000004AC0000048C0000046C000006C
:10F0800044C0000042C0000040C000003EC000007C
:10F090003CC000003AC0000011241FBECFEFD0E2F8
:10F0A000DEBFCDBF04B603FE19C080917F019091F1
:10F0B000800182349C4D91F484B7877F84BF88E1BE
:10F0C0000FB6F89480936000109260000FBE10920B
:10F0D000800110927F01E0E0F0E0099511E0A0E0EE
:10F0E000B1E0EEE7FEEF01E00BBF02C007900D922A
:10F0F000A236B107D9F721E0A2E6B1E001C01D9226
:10F10000AF37B207E1F753D1B8C67ACF8823B9F049
:10F110002091F2003091F300232B69F49091E800E4
:10F120009B7F9093E8009091E80092FD06C09EB30B
:10F130009111F9CF04C09091F1008150E7CF08956B
:10F1400030916F0120916E0190916D0180916C0161
:10F150009093640180936501C9019093620180934B
:10F16000630108951F93CF93DF93CDB7DEB7279741
:10F170000FB6F894DEBF0FBECDBF909174018091A1
:10F180006A019923D1F0843049F480916B01811197
:10F1900008C080916C018F3F21F468C0853009F46C
:10F1A000C6C08AE08093000183E080937201809161
:10F1B000EB0080628093EB00F0C0843009F456C00D
:10F1C00028F4813051F0833021F1E7C0853009F413
:10F1D000AEC0863009F4D5C0E0C010916B0112308A
:10F1E00008F0DBC0ADDF111112C080916401909175
:10F1F000650120916601A22FB0E023E0FC01A093FD
:10F200005B0020935700E89507B600FCFDCF85E032
:10F2100007C080916B01982F9D7F29F491DF89E0D1
:10F2200080930001BAC0813009F0B7C080E090E05F
:10F23000DC01ABBFFC0127912F3F69F0A093660171
:10F2400090936501809364018AE08093000185E0DA
:10F2500080937201A2C00196A11DB11D811520EFFE
:10F26000920721E0A207B10521F797C080916B01B9
:10F27000833071F581E080937301809170019091EA
:10F28000710120916C01892B61F0213009F085C05A
:10F2900090916F0180916E01909367018093680156
:10F2A0007CC0211112C082E49CED90938001809378
:10F2B0007F012CE088E190E00FB6F894A895809348
:10F2C00060000FBE2093600068C01092010165C00D
:10F2D000811163C080916C018F3F09F05EC080E0B6
:10F2E00090E0DC0123E035E0FC01A0935B0020937B
:10F2F0005700E89507B600FCFDCFFC01A0935B002A
:10F3000030935700E89507B600FCFDCF9F5FAF4FE5
:10F31000BF4F811540EF940741E0A407B10521F7E5
:10F3200081E180935700E8951092740136C080E225
:10F330008D838CED8E838BEF8F8388E589838EE1BF
:10F340008A8387E98B8382E88C8320916C0180918A
:10F350006B01811105C0FE01E20FF11D85810EC018
:10F360008130D9F4822F90E0FE01203610F4BF974F
:10F3700002C0EC55F109E80FF91F80818093690103
:10F380000CC080916B01833041F480916C0181113C
:10F3900004C080916D018093660127960FB6F894A2
:10F3A000DEBF0FBECDBFDF91CF911F91089584B70F
:10F3B000877F84BF88E10FB6F89480936000109235
:10F3C00060000FBE90E080E80FB6F8948093610073
:10F3D000909361000FBEC1E0C5BF82E085BFA5D399
:10F3E000C0936F0083E08093810078948091010145
:10F3F000882311F024D5FACF809173018111FACFBF
:10F400003CD310926F001092810081E085BF15BE41
:10F41000E0916701F091680109951F920F920FB674
:10F420000F9211240F900FBE0F901F901895CF923E
:10F43000DF92EF92FF920F931F93CF93DF93809110
:10F4400077018F77813209F0F9C180917D01909128
:10F450007E019093710180937001809178018330D7
:10F4600009F4ADC158F48130D1F0823009F0E6C121
:10F470008091E800877F8093E8000FC1853009F410
:10F48000C4C108F4BAC1863009F0D8C18091E8003F
:10F49000877F8093E80082E080930001C6C180915D
:10F4A000E800877F8093E80080917301882319F03A
:10F4B00059DE109273018091700190917101009753
:10F4C00051F12091E80022FD04C02EB32111F9CFA3
:10F4D000B5C12091F10020936A01019790937101C9
:10F4E00080937001EBE6F1E08091F2009091F300DF
:10F4F000892B81F08091F10081938091700190912E
:10F5000071010197909371018093700181E0E03760
:10F51000F80751F727DE80910001853009F0B5C06A
:10F520008091700190917101892B21F482E0809388
:10F530000001ABC08AE1EADDE0906401F090650172
:10F540008E2D8F71E3DD00916201109163010F5FD9
:10F550001F4F0E191F0980916B0181118CC0E801AA
:10F56000D695C795C70120916601A22FB0E08C0106
:10F570009D01F12CEE24E39465E0D62E73E0C72EB6
:10F58000209709F44AC04091F2005091F300452BB6
:10F59000E1F021977091F1006091F100472F562F13
:10F5A0000A01FC01A0935B00E0925700E89511244A
:10F5B000F394AC01BD014E5F5F4F6F4F7F4FDB0196
:10F5C000CA01E0E8FE120EC00FC04091E8004B7F78
:10F5D0004093E8004091E80042FDDBCF4EB341117B
:10F5E000F9CF2CC1209761F6F80120935B00D092EF
:10F5F0005700E89507B600FCFDCF209709F4C0CF6F
:10F60000FA0160935B00C0925700E89507B600FCD2
:10F61000FDCF8A019B01F12CB3CF809162019091C3
:10F620006301909365018093640181E180935700A9
:10F63000E89529C08091F2009091F300892B49F45C
:10F640008091E8008B7F8093E8008091E80082FF42
:10F6500016C0015011096091F100809164019091F0
:10F660006501FDD3809164019091650101969093AD
:10F6700065018093640101151105E1F604C08EB3A4
:10F680008111E3CFDBC080E141DD8091E8008B7F19
:10F6900093C08EB3882309F4D1C08091E80080FF25
:10F6A000F8CF80910001893091F08A3059F480912F
:10F6B0006B01813039F490916401809165019093E0
:10F6C000F10002C0809169018093F10072C0409105
:10F6D00064015091650120916201309163012F5FB7
:10F6E0003F4F241B350B80916B01811135C0CA013E
:10F6F00040916601A42FB0E036952795211531057C
:10F7000011F14091F2005091F3004032510569F43B
:10F710004091E8004E7F4093E8004091E80040FDB2
:10F7200004C04EB34111F9CF89C0ABBFFC01479172
:10F7300056914093F1005093F1000296A11DB11D26
:10F7400021503109DBCF8091620190916301909348
:10F750006501809364012AC0823041F5E901209758
:10F7600029F18091F2009091F300809769F48091E3
:10F77000E8008E7F8093E8008091E80080FD04C05F
:10F780008EB38111F9CF5AC08091640190916501C7
:10F790005ED38093F10080916401909165010196A0
:10F7A00090936501809364012197D9CF82E0809383
:10F7B00000018091E8008E7F8093E80036C0809140
:10F7C000E800877F8093E8008091E80080FD04C016
:10F7D0008EB38111F9CF32C0809172018093F10014
:10F7E0001092F1001092F1001092F100809100014E
:10F7F0008093F1001092F100DCCF8091E800877FC8
:10F800008093E8001092720110C08091E800877F19
:10F810008093E8008091E80080FD04C08EB38111E0
:10F82000F9CF0CC0809100014FCFDF91CF911F9194
:10F830000F91FF90EF90DF90CF9000C1DF91CF91BB
:10F840001F910F91FF90EF90DF90CF900895292F97
:10F8500030E02230310539F02330310549F02130D4
:10F86000310561F410C08BE190E024E331E01EC06B
:10F87000882371F0813089F08230A1F080E090E03F
:10F8800020E030E013C082E190E02FE431E00EC0D0
:10F8900084E090E020E331E009C088E190E026E1D7
:10F8A00031E004C082E190E022E031E0FA013183EE
:10F8B0002083089507B600FCFDCFF999FECF23E021
:10F8C000FB0180935B0020935700E89507B600FC8E
:10F8D000FDCF81E180935700E895089507B600FCBD
:10F8E000FDCFF999FECF25E0FB0180935B002093CB
:10F8F0005700E89507B600FCFDCF81E180935700E3
:10F90000E895089507B600FCFDCFF999FECF21E0F8
:10F910000A01FB0180935B0020935700E8951124B6
:10F92000089521E2FC01209357008491089529E075
:10F93000FC012093570084910895E1E0F0E089E014
:10F94000809357008491089507B600FCFDCFF99984
:10F95000FECF809599E0E1E0F0E0082E909357000B
:10F96000E895089520917D0130917E012617370793
:10F9700048F06115710539F42091E8002E7F20933D
:10F98000E80001C0B901FC0120E06115710591F1A9
:10F990008EB38823E1F18530E1F18091E80083FDA9
:10F9A0003AC08091E80082FF06C08091E80082FFA3
:10F9B00024C080E008958091E80080FFE6CF809128
:10F9C000F2009091F3006115710551F080329105BC
:10F9D00038F421912093F100615071090196F3CF21
:10F9E00021E0809709F020E08091E8008E7F8093ED
:10F9F000E800CBCF2111CCCFD8CF8EB3882339F0FC
:10FA0000853039F08091E80083FFCFCF04C082E0D9
:10FA1000089583E0089581E00895EBEEF0E08081A1
:10FA200081608083EDEEF0E010826093EC00408313
:10FA30008091EE00881F8827881F089580917701A4
:10FA400087FD05C08091E80080FF0DC010C0809147
:10FA5000E80082FD04C08EB38111F9CF0895809132
:10FA6000E8008B7F07C08EB38111ECCF08958091A1
:10FA7000E8008E7F8093E800089565D06CD0E0EEBA
:10FA8000F0E0808181608083E8EDF0E080818F7715
:10FA9000808319BCA7EDB0E08C918E7F8C93808120
:10FAA0008F7E80831092760108950F931F93CF93DA
:10FAB000DF9349D050D0C8EDD0E088818F7788831C
:10FAC00088818068888388818F7D8883E7EDF0E076
:10FAD00080818068808319BC1EBA1092750100EE87
:10FAE00010E0F80180818B7F80838881816088832A
:10FAF00042E260E080E091DFE1EEF0E080818E7F25
:10FB00008083E2EEF0E08081816080838081886084
:10FB10008083F80180818E7F8083888180618883E3
:10FB2000DF91CF911F910F910895E8EDF0E0808172
:10FB30008F7E8083E7EDF0E080818160808381E0CB
:10FB400080937601B2CFE8EDF0E080818C7F8083F6
:10FB50001092E20008951092DA001092E1000895E8
:10FB60001F920F920FB60F9211240BB60F922F9384
:10FB70003F934F935F936F937F938F939F93AF9335
:10FB8000BF93EF93FF938091DA0080FF1BC08091B9
:10FB9000D80080FF17C08091DA008E7F8093DA0052
:10FBA0008091D90080FF0BC084E189BD86E189BDC9
:10FBB00009B400FEFDCF81E08EBB40D103C019BC6B
:10FBC0001EBA3CD18091E10080FF17C08091E20015
:10FBD00080FF13C08091E2008E7F8093E2008091CD
:10FBE000E20080618093E2008091D800806280937F
:10FBF000D80019BC85E08EBB21D18091E10084FF43
:10FC00002EC08091E20084FF2AC084E189BD86E194
:10FC100089BD09B400FEFDCF8091D8008F7D80930F
:10FC2000D8008091E1008F7E8093E1008091E20016
:10FC30008F7E8093E2008091E20081608093E200F9
:10FC400080917501882311F084E007C08091E30062
:10FC500087FF02C083E001C081E08EBBEFD08091BE
:10FC6000E10083FF21C08091E20083FF1DC08091ED
:10FC7000E100877F8093E10082E08EBB10927501E6
:10FC80008091E1008E7F8093E1008091E2008E7F81
:10FC90008093E2008091E20080618093E20042E282
:10FCA00060E080E0BADECAD0FF91EF91BF91AF91E2
:10FCB0009F918F917F916F915F914F913F912F9184
:10FCC0000F900BBE0F900FBE0F901F9018951F93B3
:10FCD000CF93DF9300D0CDB7DEB7E7E7F1E08091B7
:10FCE000F100819381E0EF37F807C9F7A0DB80913D
:10FCF000E80083FF8FC09091770180917801863072
:10FD0000E1F128F4882351F08530B1F083C08830C8
:10FD100009F453C0893009F462C07CC09D7F9038DB
:10FD200009F078C08091E800877F8093E800109206
:10FD3000F1001092F1004CC091116CC0109179014A
:10FD40001F778091E3008078812B8093E30080917E
:10FD5000E800877F8093E80071DE8091E80080FFF3
:10FD6000FCCF8091E30080688093E300112311F0C1
:10FD700083E001C082E08EBB4DC09058923008F005
:10FD800049C0AE014F5F5F4F60917B018091790167
:10FD900090917A015CDD009709F43CC02091E80065
:10FDA000277F2093E800BC0189819A81DBDD809167
:10FDB000E8008B7F8093E8002DC0903859F5809142
:10FDC000E800877F8093E800809175018093F100BF
:10FDD0008091E8008E7F8093E80030DE1BC0911197
:10FDE00019C0909179019230A8F48091E800877F42
:10FDF0008093E8009093750121DE80917501811157
:10FE000004C08091E30087FF02C084E001C081E06C
:10FE10008EBB14D08091E80083FF0AC08091E80077
:10FE2000877F8093E8008091EB0080628093EB00F5
:10FE30000F900F90DF91CF911F91089508958EB389
:10FE4000882321F08091E80083FD41CF0895F9993E
:10FE5000FECF92BD81BDF89A992780B50895262FCF
:10FE6000F999FECF1FBA92BD81BD20BD0FB6F8949F
:0EFE7000FA9AF99A0FBE01960895F894FFCF02
:10FE7E00020112034C0055004600410020004400D0
:10FE8E0046005500000018034400650061006E0036
:10FE9E002000430061006D006500720061000000EB
:10FEAE000403090409021B00010100803209040049
:10FEBE000000FE0102000921030000000C100112D7
:10FECE0001100100000020EB03FB2F0000010200D7
:02FEDE00010021
:10FFA00089CC9CCCAFCCBDCCC2CCC7CCCDCC089539
:08FFB0000895089508950895D5
:10FFE000DFCFDFCFDFCFDFCFDFCFDFCFDFCFDFCFA1
:08FFF000DFCFDFCFDFCFDFCF51
:08FFF80000F0010010DFFBDC4A
:040000031000F000F9
:00000001FF
